:020000040800F2
:10500000981A0020D5500008F1820008197B00088A
:105010000000000000000000000000000000000090
:10502000000000000000000000000000B18F000838
:1050300000000000000000005D880008CD9000081E
:10504000E7500008E7500008E7500008E750000864
:10505000E7500008295B0008E7500008E750000807
:1050600000000000E7500008515A0008E75000080F
:10507000E75000086D7F000800000000E7500008BE
:1050800000000000E75000080000000000000000E1
:10509000E750000800000000E7500008E750000853
:1050A000E7500008E7500008E7500008599800084A
:1050B000E7500008E7500008000000000000000072
:1050C0000348854600F060FC0048004785A60008BC
:1050D000981A00200448804704480047FEE7FEE78E
:1050E000FEE7FEE7FEE7FEE769910008C150000811
:1050F00030B50B46014600202022012409E00D4670
:10510000D5409D4205D31D469540491B25469540F7
:1051100040191546521E002DF1DC30BDF0B51FB40C
:105120000646002082B005464024019100901BE015
:10513000019922460F46304600F04EFB049A059B2B
:10514000801A994110D310461946224600F034FBCC
:10515000361A8F410197224601200021009F00F05E
:105160002BFB38184D4100902046641E0028DFDCE0
:10517000019B00982946324607B0F0BD03460B4319
:105180009B0703D009E008C9121F08C0042AFAD2FD
:1051900003E00B780370401C491C521EF9D2704783
:1051A000D2B201E00270401C491EFBD270470022BF
:1051B000F6E710B513460A4604461946FFF7F0FF16
:1051C000204610BD30B504460020034600E05B1CBD
:1051D000934203D2E05CCD5C401BF8D030BDF8B503
:1051E00002464A40D40F42004B0052085B089A42E4
:1051F00002D20246084611464A0023D0C30D4A0097
:10520000DDB2120EAD1A202D35DA49020126490A07
:10521000F6058A19002C00D0524220214F1B11465E
:10522000B9402A411018C20D9A4221D0002C17D043
:10523000012D08DCDA05801AD20F8019D207DBB203
:1052400000F0F6FAF8BDDA05801A012340001B06CB
:10525000C01880185A428018CA0F1043490007E04E
:105260004908C2071143DA05801A801940088018DE
:1052700000F0D6FAF8BD61000122511A001BF7E7D1
:105280000122D2075140AAE70122D2075040A6E7E7
:1052900070B502464A40D50F40004A00ED0740086D
:1052A0005208002814D0002A12D0C40DD30D410298
:1052B0000120C0055202490A520AE41A09181218BC
:1052C0007D34914201D3641C00E04900002C01DAD6
:1052D000002070BD0023914201D3891A0343400886
:1052E00049000028F7D100290AD0914202D10121BA
:1052F000C90705E0914201D2012101E00121C94322
:10530000E005C018401900F08BFA70BDF0B50746F3
:105310000846584087B0C00F049048000E46590018
:1053200040084908BC1A884105D2384631461E4615
:1053300017460B4602465800400810434CD0300D2B
:10534000039040055900400D490D0590401A029008
:10535000402872DA18030121000B09050843019067
:1053600004980092002805D00199524200208841FB
:1053700000920190029840210A1A0199009800F0C9
:105380001BFA05460C466B4607CB00F036FAC019EF
:105390007141039A0E0D0023D71756401A467A40E2
:1053A000164344D0049A002A2DD0029A012A039A67
:1053B00015DC1205C01A914101263605001C714109
:1053C000D20F059ED2070093019202962A462346E9
:1053D00000F074FA07B0F0BD38463146FAE716051A
:1053E000224A0F46B218C01AB74101210905001C14
:1053F0004F4100187F41114618187941E20F1043C0
:105400006D19644113E0E2076D0815436408C20793
:105410001443039A01261205C01A91413605001C57
:105420007141CE07400830434908C01851412A460F
:10543000234600F036FACDE7FFE70498012240004A
:10544000C117121A00238B4104983146C417381A29
:10545000A141EEE730B40124E407634030BC55E7D6
:1054600030B40124E407614030BC4FE70000E0FFA6
:10547000F0B51FB488B00B990998002448400999E9
:10548000C00F490049080991C0070B9900904900D5
:1054900049080B9109990898A64608431CD00B9916
:1054A0000A98084318D0099801244000420D48008A
:1054B000410D099824050003000B204309900B9827
:1054C0000003000B20430B9050181C494018002289
:1054D00001901446104605E0002001460DB0F0BDD5
:1054E000032801DA034600E003239C46C11A0AAEF2
:1054F0000AE05F0008ADED5B4F00F75B7D430027DE
:10550000AA187C41491C5B1E6145F2DD410004ABD9
:105510005A522104120C0A43240C401C0828DFDBD9
:10552000019802900099704601910090059B049AA1
:105530000799069800F0C2F9D0E700000DFCFFFFC4
:10554000F0B50C465C4085B0E40FE40703944C00D2
:1055500000266408590094464908024602962243F0
:1055600021D062460A431ED06200570D4A000E0346
:105570002303550D012402462C492405781B1B0BDF
:10558000360B401823432643614600901C46501AB0
:10559000B44103D30098401C009002E09218009898
:1055A0005B41002803DA0020014605B0F0BD002071
:1055B000012109050746864611E064461D46141B75
:1055C000B54106D36546521BB341744607430C43AD
:1055D000A646CD0740084908284392185B41054676
:1055E0000D43EAD11046184313D060461946504087
:1055F0007140084306D06046101AB34106D201221A
:10560000002306E000220123DB0702E00122D2434F
:105610005310009874460105381C6141029C039D9B
:105620000019694100F03DF9BFE70000FD030000EB
:10563000C217C10F504010B54018CA079623002169
:1056400000F0F6F810BD10B500229623114600F0C8
:10565000EFF810BD0EB5C217C10F5040CA07401871
:105660000021054B0293019200910A460B4600F07F
:1056700025F903B000BD0000330400000EB5054954
:105680000291002100910A460B46019100F016F9A3
:1056900003B000BD33040000410040020122400A73
:1056A000D205090E80187F2901DA0020704796295B
:1056B00003DC9622511AC8407047963988407047DB
:1056C00070B5CD0F4A0009030123090B1B051943CF
:1056D0000B4BED070024520D9A4201DA002070BDF9
:1056E000074B34339A4203DC9A1A00F075F802E053
:1056F0000449511888402C43F1D0404270BD00004D
:10570000FF030000CDFBFFFF4A0009030123090B43
:105710001B051943094B10B5520D9A4201DA0020BE
:1057200010BD064B34339A4203DC9A1A00F054F849
:1057300010BD03495118884010BD0000FF03000050
:10574000CDFBFFFFC20FD207400040080BD0C10DB8
:105750000723DB01C91840020905400A1143C208AA
:10576000400711437047002001467047CB0FDB070D
:10577000490010B5490802460A4307D00A0D07241C
:105780000903E401090B121B002A01DC002010BDF3
:10579000C900440F0C43C100E018D205801800F086
:1057A0003FF810BD0122D207002800DB101A0029A3
:1057B00000DB511A8142704710B5202A04DB0146F4
:1057C000203A9140002010BD914020239C1A0346AE
:1057D000E3401943904010BD10B5202A04DB084671
:1057E000203AD040002110BD0B46D340D0402024A9
:1057F000A21A91400843194610BD10B5202A06DBB5
:10580000CB170846203A1041C1170B4306E00B4660
:105810001341D0402024A21A91400843194610BDDC
:10582000002904DA401C490001D1400840007047BB
:1058300070B40024050C05D11024000402D1002905
:1058400021D01124050E01D100020834050F01D129
:105850000001241D850F01D18000A41C002801DB5C
:105860004000641C002908D020252E1B0D46F54061
:10587000A14000D001212943084301061B1B000A57
:10588000DB1D02D5002070BC7047DB05181880189E
:105890000029F8DA401C4900F5D170BC40084000EE
:1058A000704710B5002B08DA0024401C61419218A3
:1058B0005B411A4301D14008400010BDF0B51FB450
:1058C00082B005460C0003D0084604F085F802E0DB
:1058D00004F082F820300246009021462846FFF767
:1058E0006BFF049B059A04460F4618431143084377
:1058F00014D0184610431BD0009840210A1A1846AD
:105900000599FFF769FF05460E46009A0599049828
:10591000FFF752FF084305D0012004E02046394636
:1059200007B0F0BD0020C11705430E432C43374399
:1059300000990E986305401A7905E40A00220C4389
:10594000FD0A0A3002D500200146E9E701051019D9
:1059500069410C9C0D9D00196941FFF7A2FFDFE72B
:1059600010B5002904DB0124E40740428C412146A4
:10597000002B04DB1C460123DB075242A341994262
:1059800000D1904210BD0000064C0125064E05E0F6
:10599000E36807CC2B430C3C98471034B442F7D350
:1059A000FFF792FBF8A9000818AA000838B50446CA
:1059B000064805490068FFF79BFB604300E0401E76
:1059C00000900028FBD138BD40420F001C01002090
:1059D000F8B50446006881688907890F012902D15A
:1059E0000168C90722D18168114A1026114001259A
:1059F00000290ED18168294381600120FFF7D6FF7D
:105A000000F07AFF07460CE000F076FFC01B0A2882
:105A100007D9606D30436065A06D2843A065012003
:105A2000F8BD20680068C043C007EDD10020F8BD74
:105A30001700008010B500231A4603E0845CE318C9
:105A40009BB2521C8A42F9D3D84380B210BD0000E9
:105A500010B5034800F010FD024800F00DFD10BD28
:105A600038160020F015002030B5446C1C252C4061
:105A70000125A540046C6560046863608368102B91
:105A8000036803D099600068C26030BD9A60006806
:105A9000C16030BD1449012048720A4602205E32BE
:105AA000507203203C3A507204200E3A50720F4854
:105AB0000D4B0078087022310870203108770C49AE
:105AC0005A1C0878587149789971233318715971A3
:105AD000203318775977107551751A461E32107594
:105AE000517510765176704750110020D700002074
:105AF000F400002010B503F033FA202003F0DCFAA4
:105B0000012004F019FB002003F0D6FA044804F049
:105B1000B7F9044804F066FC002004F09BFC10BDBB
:105B2000C000002083800000F8B505200121000797
:105B300000F0D2FE0025184C002800D06560174EFA
:105B40000221304600F0C8FE00281DD1012020703F
:105B50001348808F00280ED00127BF02002239464B
:105B6000304600F0C2FE0A2004F03CF9012239461A
:105B7000304600F0BAFE0B48656000880A214843B1
:105B80000949088003F07AFE012000F0DDFD0220C3
:105B900000F0DAFDF8BD00000C0100200004005008
:105BA000500D0020E4000020F000002070470000AD
:105BB00010B5084900224A6107494B684C15234338
:105BC0004B604B68082423434B60C009C00102604E
:105BD00010BD000080160020002002407FB5002587
:105BE0000C460646039500F07FFDE009029003A9EC
:105BF00001960095684600F00FFD002804D000F0E3
:105C000047FD002004B070BD00F042FD0120F9E71F
:105C100010B5002302E0C45CCC545B1C9342FAD361
:105C200010BD000010B5214A00219069C30520482D
:105C300004D54169022319434161911593699B057C
:105C400005D54369012423434361630219439369E2
:105C50005B0505D54369082423434361E3011943E8
:105C600093691B0505D543690424234343616302FB
:105C7000194393699B0405D5436910242343436169
:105C80006302194393699B0304D5446920231C4391
:105C9000446119439369DB0305D5436940242343D9
:105CA0004361A0020143916110BD00000020024049
:105CB0008016002070B5054600F01EFE0646184C02
:105CC0000AE0681C08D0002D04D000F015FE801BEF
:105CD000A84201D9032070BDA069C007F1D1A06915
:105CE000800701D50220A061A069C00511D4A06978
:105CF00080050ED4A06940050BD4A069000508D426
:105D0000A069800405D4A069800302D4A069C003FF
:105D100003D5FFF787FF012070BD002070BD000094
:105D200000200240F8B51746002605460C4600F054
:105D3000DBFC09E029460220226800F0B7FC0028BD
:105D400004D1241D2D1D361DBE42F3D300F0A0FC4E
:105D5000BE4201D20020F8BD0120F8BD10B50849AF
:105D600002460020054B497905E044001C5B944243
:105D700003D0401CC0B28842F7D310BD7812002077
:105D80005800002010B500F0ACFD10BD10B509485A
:105D900000F0D4FF80B2FFF771FC074A074BFFF712
:105DA00067FB0022064BFFF7CBFBFFF7ADFC80B291
:105DB00010BD0000E8140020F853E3A59B843E408A
:105DC00000408F4070B5324930488A7F0275C97FE4
:105DD000417530490A780276497841762B49052089
:105DE000133148720A2004F0EDFA7D20C00004F05F
:105DF00003FB2649002213310C2004F0CDFB0021C7
:105E00000C2004F0DBFB022004F02CFB224C204D84
:105E100000210F2004F056FA20422863F8D0286BA6
:105E2000411C30D040042DD58122D20100210F2009
:105E300004F087FB0021102004F044FA41061348C7
:105E4000490E0022633004F073FA104C6334607A18
:105E5000052817D102220F49601DFFF7B3F900286A
:105E600010D10B48A67C6E710422611C4430FFF7F0
:105E700085F921461331084672005130FFF77EF94B
:105E80000320287070BD02F057FA0000B111002005
:105E900058000020F400002000D0272410B5084846
:105EA00000F096FA0A21064800F032FA044800F0A1
:105EB0001DF9800503D5024800F01AF980B210BD23
:105EC0008C140020F8B52F4D00220121284600F047
:105ED0000CFDFFF7E3FFFFF7B6FB2B4E3146FFF754
:105EE000D7F92A4C0122A0601146284600F0FDFC9B
:105EF0002749A068002588423EDB2078254F0028EE
:105F000015D02570FFF7CAFFFFF79DFB3146FFF75D
:105F1000BFF9A060FFF716FC00223B46FFF79AFA94
:105F200000221D4BFFF7A4FAFFF720FC6060A06879
:105F3000FFF708FC00223B46FFF78CFA174A184B84
:105F4000FFF796FA06460F466068FFF7FBFB134A19
:105F5000144B5242FFF78CFA32463B46FFF7D6F914
:105F6000FFF704FC10496060884201DD616004E0D5
:105F7000FF21C905C84200D365606068FFF78CFB4C
:105F8000C0B2F8BD0004005000401B4430000020A7
:105F90000000604000000C4000E0644033333333C5
:105FA00033B33040CCCCEC3F0000C842F8B50546D6
:105FB00004464035287C0026012808D0012028749A
:105FC000206881688907890F01290ED101E002202C
:105FD000F8BD0168C90708D0606D202108436065DD
:105FE0000126002028743046F8BD616DFF22013281
:105FF0009143022211436165C1688907890F0091AD
:10600000C16889088900C1602068816892071143CE
:10601000816000F071FC07460EE000F06DFCC01BD3
:106020000A2809D9606D0221884310210843606560
:10603000002028740120F8BD206880680028ECDB6F
:106040002068C168009A1143C160606D80088000BB
:10605000401C6065C5E70000F8B506460D464036B1
:10606000317C01290DD00121317401688A68520701
:1060700009D5416D20221143416500203074012073
:10608000F8BD0220F8BD174B6A68D80547109A4240
:10609000154C8A6A2B6812D05B035B0B1A438A6229
:1060A0002968490305D5A1680143A1600A20FFF7CB
:1060B0007DFC2868800312D5A06838430EE05B039E
:1060C0005B0B9A438A622968490302D5A168814320
:1060D000A1602868800302D5A068B843A0600020B2
:1060E0003074F8BD0110000000270140406D70477A
:1060F0000068006C7047000070B5040006D0606D49
:10610000264600254036002802D006E0012070BD5A
:10611000A5653574204600F0D3F8606DC00603D441
:1061200021688868400705D5606D102108436065C7
:106130003574EBE7606DFF22013290430222104379
:10614000606588688207920F5B48012A02D10A685D
:10615000D2072BD1032362689B079A4205D05B428A
:106160009A4202D05B009A4209D10A6992009208D1
:106170000A6121680A6963681A430A610CE00A69C6
:10618000920092080A6181680F2292049143816013
:1061900081686268114381602168CA6818239A4344
:1061A000CA602168CA68A3681A43CA60816801226C
:1061B0005206914381608168A28E5206114381602C
:1061C00020688168C90004D4816801221207114344
:1061D00081602068C168394A1140C1602069E16866
:1061E000022825D000200143204620300278037B7E
:1061F00052035B001A431143226B1143A2699203BD
:106200001143E269D20311432268D3681943D16074
:10621000616A0A46FF3AC23A05D0A26A114322686F
:10622000D3681943D16042780121012A02D00BE0E2
:106230000420D8E70078002823D0606D2022104386
:106240006065A06D0843A065E06B012820681FD041
:106250000169C90703D00169490849000161206843
:106260004169C908C900416120684169A26B1143B5
:106270004161A565606D80088000401C606500205C
:1062800070BD2068C26801231B041A43C260DBE7AB
:106290000269FF239B009A43026120680269236C14
:1062A000A66C1A43636C33431A4302612068026987
:1062B0000A430261D3E70000002701401902FEFFF4
:1062C00010B586B0044614216846FEF770FF0E49EB
:1062D0002068884216D10D48416B42151143416335
:1062E000C16A01221143C162C06A6946104005902B
:1062F000022000900320019000200290052000075A
:1063000000F02EFA06B010BD00240140001002403B
:10631000F8B504464069254640350E4608280BD09E
:106320002068C068C00709D0606D202108436065FF
:10633000002028740120F8BD082700E00C2700F099
:10634000DBFA009011E0701C0FD0002E05D000F099
:10635000D3FA0099401AB04207D9606D042108436E
:106360006065002028740320F8BD2068006838426A
:10637000E9D0606D01214902084360652068C16869
:1063800009058A0F0C21002A1BD12022125D002A48
:1063900017D10268120714D5826853070122002B17
:1063A00008DB43688B434360606D130298431043DE
:1063B000606506E0606D202318436065A06D1043A2
:1063C000A065A069002801D1206801600020F8BD07
:1063D00070B50446216800208968490721D4254604
:1063E0004035297C01291CD001212974E16901294A
:1063F00004D02046FFF7ECFA002811D1616D0A4A5B
:106400001140FF220132114361650021A165297409
:1064100022681C21116021688A6804231A438A605B
:1064200070BD022070BD0000FEF1FFFF70B50024BA
:10643000014620314A79022A03D00421C163012494
:1064400018E0026813680E25AB43136002681368F6
:106450005B085B001360436C1C221340012215464D
:106460009D40036C5D604A7100220A71816B0029B6
:1064700000D08847204670BDF0B4016C0D680168FB
:106480000C68466C1C2304221E401746B7402F425E
:106490000ED067070CD50C68A40602D40C68944390
:1064A0000C60416C19408A40016C4A60016B1AE033
:1064B0000227B74002462F402032002F17D0A707EF
:1064C00015D50C68A40605D40C680A25AC430C60ED
:1064D00001215171446C02211C40036CA1405960A0
:1064E00000211171C16A002918D0F0BC08470827A3
:1064F000B7402F4212D0240710D50C680E25AC43AC
:106500000C60446C01211C400B46A340046C63608A
:10651000C163517100211171416BE4E7F0BC704718
:1065200070B504003CD01F48256814212818FEF7D8
:10653000DFFD800060641C4820640221204620307A
:106540000246417129681948E3680140A0686669FC
:106550001843236933431843A3691843E369184375
:10656000236A1843084328600121A06889038842F0
:1065700010D00D488030836A656C1C210D400F26B9
:10658000AE40B3438362656C63680D40816AAB4083
:106590000B4383620020E06301215171107170BDD3
:1065A000012070BDF8FFFDBF000002400F80FFFF1B
:1065B000F8B504468C46203001790025012909D020
:1065C0000126067141790027012905D007710225AE
:1065D0002846F8BD0220F8BD02214171E76320681A
:1065E000016849084900016061462046FFF73CFA0E
:1065F000206B00282068016801D00E2205E00422EB
:1066000091430160206801680A22114301602068FB
:10661000016831430160DBE7F8B51A4E0546307C6E
:106620000F46012807D0012030741748FFF742FBBE
:10663000010002D021E00220F8BD0020C0433860F4
:106640006C6814E02046FFF7B3FA0F48FFF732FBFF
:1066500001460E48426808239A4342604268431547
:106660009A434260002901D03C6006E08034A8686B
:106670006A68C0018018A042E4D80020307408463F
:10668000F8BD00008016002050C30000002002402A
:1066900005484168022211434160416801221143CB
:1066A000416000207047000000200240F8B50C4C0B
:1066B0001646207C0F46012808D001202074094886
:1066C000FFF7F8FA0025002802D006E00220F8BD06
:1066D00065613E600348FFF7EDFA2574F8BD0000E0
:1066E0008016002050C3000011484168C9070BD034
:1066F000EFF3108172B60F4AC2600F4AC26081F395
:1067000010884168C9070ED1416889070DD5EFF39C
:10671000108172B6094A0261094A026181F3108848
:106720004068800701D501207047002070470000B5
:1067300000200240EFCDAB8905040302BFAE9D8C63
:10674000161514137047000010B504494A69024237
:1067500002D04861FFF7F6FF10BD000000040140C1
:10676000F8B500230124A2E027469F403A4070D0AC
:106770004D68022D01D0122D14D1DD08AD002D1869
:1067800000952D6A5E07AC46F50E0F26AE46AE406C
:106790006546B543AC460E697546AE4065462E4328
:1067A000009D2E624D68012D05D0022D03D0112DC4
:1067B00001D0122D16D185680326AC465D00AE4689
:1067C000AE406546B543AC46CE687546AE406546BC
:1067D0002E43866046680D79BE43ED06ED0F9D4061
:1067E0003543456006685F000325BD40AE46AE43B5
:1067F0000D79B446AE07B60FBE4065462E4306601F
:10680000C6687546AE438D68BD403543C5604D686A
:10681000ED004BD5294D6E6B26436E639E08284DC7
:10682000B6007519AC46AD689E07360F0F27B74006
:10683000BD4305273F07B84201D1002715E0214F8E
:10684000B84201D1012710E01F4FB84202D1022700
:106850000BE02BE01D4FB84201D1032705E01C4F90
:10686000B84201D1052700E00627B7402F4365460F
:10687000AF60184D2E684F689643FF0300D516434E
:106880002E606E684F689643BF0300D516436E6056
:10689000AE684F689643FF0200D51643AE60EE68BF
:1068A0004F689643BF0200D51643EE605B1C0A6832
:1068B0001546DD4000D057E7F8BD0000001002404B
:1068C000000001400004005000080050000C00507F
:1068D000001C0050000401400069084000D0012065
:1068E000704742694A4042617047002A01D0816185
:1068F00070478162704700000148006870470000DF
:106900001801002002480168491C0160704700001E
:106910001801002010B508480024016840221143E6
:106920000160204600F00AF8002801D0012401E0AF
:1069300000F030FA204610BD0020024070B5054638
:1069400009487D210024C9000068FEF7D1FB00F052
:10695000C5FE002801D0012404E000222946501E73
:1069600000F038FA204670BD1C01002070477047C7
:10697000F8B5664CA078401CA07001202071E08A18
:10698000401CE0826248008802F050FB6148C088E9
:10699000FEF759FE6049FEF77BFC604D2968FEF763
:1069A0001EFC28606078002500280BD102215C487D
:1069B000FFF792FF02005B495B4819D00022FFF706
:1069C00094FF2563594E01203768C005874257DB85
:1069D000208AFEF738FE01467F20C005FEF758FCEE
:1069E0003946FEF751FC306051480221017049E000
:1069F0000122D1034C48FFF778FF4648C088FEF7D4
:106A000022FE4549FEF744FC216BFEF7E8FB4949AD
:106A100020638842D6DD3F480127F92640300090A8
:106A20000A213046FEF764FB002903D13D493E4868
:106A3000FFF7A8F902213A48FFF74EFF002801D0DE
:106A4000002701E0002F12D102213548FFF744FF53
:106A500000280CD103F0E0FE00990120888003F0AB
:106A60003BFF642003F0BEF934493348C8600A2074
:106A700003F0B8F93046761EF6B20028D0D1A1E76F
:106A80002B48057002212648FFF726FF002809D071
:106A90002563224E2A4937682A488F4214DD012196
:106AA000017012E01B48C088FEF7CDFD1A49FEF7C1
:106AB000EFFB216BFEF793FB234920638842E8DB61
:106AC0001E491D48C860E4E705701248408F401E0B
:106AD000FEF7AEFD3946FEF765FE06D86079002860
:106AE00003D01A490120087001E0184805700948D0
:106AF000408FFEF7A8FD3168FEF754FE04D260799E
:106B0000002801D003F04CFEF8BD0000D4000020A6
:106B100074000020500D002000007A441001002075
:106B2000000400500080000000000050140100200C
:106B30006A000020000040400400FA0500ED00E07B
:106B40000000F0425E0000200000A0406C00002029
:106B5000704770B505000DD002202C462034A0737C
:106B6000284601F00BFA284600F0BEF80020A0737A
:106B7000607370BD012070BD7047704710B504464A
:106B800000680168C943C90708D18168C943C907BA
:106B900004D1012141602046FFF7EAFE2068016828
:106BA000C943890708D48168C943890704D40221ED
:106BB00041602046FFF7DAFE20680168C9434907B3
:106BC00008D48168C943490704D4042141602046A0
:106BD00000F0DEF820680168C943090708D481681D
:106BE000C943090704D4082141602046FFF7B0FFDC
:106BF00020680168C943C90608D48168C943C90629
:106C000004D4102141602046FFF7B1FE20680168DE
:106C1000C943890608D48168C943890604D4202160
:106C200041602046FFF7A9FF20680168C943490673
:106C300008D48168C943490604D4402141602046F4
:106C4000FFF79AFF10BD0000F8B5040005D02546F7
:106C50002035A87B002802D006E00120F8BD0020E6
:106C60006873204600F052F80220A8732068C268BA
:106C700084466368012B04D00120A16AC0058142CB
:106C800001D11E20824315486169814201D0144818
:106C900002401448A668024018463043676A266AD4
:106CA0003E433043A66A30431043012B03D00122F8
:106CB000D205964203D12369E2681A431043074A7A
:106CC000914205D0A2691143E2690243084610438C
:106CD0006146C8600120A8730020F8BDFFFF0000D6
:106CE0003F1FFFFFF8F119FF10B500680549884202
:106CF00007D10548816B4900490881630D2000F0E8
:106D000055F810BD007C00400010024010B500682E
:106D1000084988420CD10848816BC2041143816341
:106D2000002201210D2000F055F80D2000F048F858
:106D300010BD0000007C0040001002400068C069E7
:106D40007047000070B50224034620339C730F4C3B
:106D50002568E604354325600468E568B6123543C6
:106D6000E5600568AE6801242643AE6005682E69BB
:106D700026432E610568A96101684A6100680169BE
:106D80000422114301619C73002070BD0004014086
:106D9000704700000448416B012211434163816B3D
:106DA000020411438163704700100240C106C90EFE
:106DB00001208840014908607047000080E100E040
:106DC000C106C90E012088400149086070470000D3
:106DD00000E100E010B501F08DFA10BD02494A68EB
:106DE00082434A607047000000700040024801681A
:106DF00082151143016070470070004002494A68E3
:106E000002434A6070470000007000400548016876
:106E10000222114301600448016904221143016107
:106E200030BF70470070004000ED00E00A4B1A6868
:106E30009208920002431A6008480369042213432F
:106E40000361012906D040BF20BF20BF01699143E3
:106E50000161704730BFF9E70070004000ED00E0CD
:106E6000F8B504460078544D800672D5524E00277E
:106E7000403EB06BC00004D4B06BA9050843B063BA
:106E800001274E480168C90511D4016882151143D4
:106E90000160FFF731FD009005E0FFF72DFD00993F
:106EA000401A642837D845480068C005F5D53268CF
:106EB0000321090560680A400140914208D081031E
:106EC000890F032904D13168890301D50120F8BD58
:106ED0002A69032109040A4022D0084090421FD0A9
:106EE000207880061CD528692A6988430121C904B5
:106EF0000A432A612A698A432A612861C0050FD59D
:106F0000FFF7FAFC009008E0FFF7F6FC0099411A41
:106F10002B48814201D90320F8BD28698005F3D5AB
:106F200061688803800F032805D132680005824319
:106F300001400A433260286903226168120411404B
:106F400008432861002F04D0B16B01200007814362
:106F5000B1632078C00705D0E868A1688008800088
:106F60000843E8602078800705D5E8680C2188434D
:106F7000E1680843E8602078400706D5E868032107
:106F80008902884321690843E8602078000706D514
:106F9000E86803210903884361690843E8602078B1
:106FA000000606D5E868032189048843A1690843DF
:106FB000E8600020F8BD0000401002400070004072
:106FC00088130000F8B50E4605007DD053480068D0
:106FD000C007C00FB0420AD25048016849084900B2
:106FE000314301600068C007C00FB04271D12878FA
:106FF0004B4C800705D5E068F0218843A968084319
:10700000E0602878C00752D06868022817D00328AB
:1070100018D02168012818D08905002959DAE168BB
:10702000890889000143E160FFF766FC696807464B
:10703000022912D003291CD0012926D033E021686F
:107040008903EAE721688901E7E74907E5E7FFF7F0
:1070500053FCC11B3348814223D8E0680007800FEE
:107060000228F4D123E0FFF747FCC11B2D488142E1
:1070700017D8E0680007800F0328F4D117E0FFF766
:107080003BFCC11B274881420BD8E0680007800FFA
:107090000128F4D10BE0FFF72FFCC11B21488142EE
:1070A00001D90320F8BDE0680007800FF3D11B4829
:1070B0000168C907C90FB1420DD9016849084900E3
:1070C00031430160006800E003E0C007C00FB04238
:1070D00001D00120F8BD2878400706D5E0680721D7
:1070E00009028843E9680843E0602878000707D56B
:1070F000E0680721C90288432969C9000843E060A4
:1071000000F036F8E168084A0906090F515CC840EA
:10711000064908600020FFF711FCF8BD002002407E
:107120000010024088130000D6A900081C010020AE
:10713000044805490068C968044A4905490F515C7B
:10714000C84070471C01002000100240EFA9000851
:10715000044805490068C968044A8904490F515C1C
:10716000C84070471C01002000100240EFA9000831
:1071700010B5184AD1680C20084004280BD0082804
:1071800010D00C2810D050680004410F0120C0031B
:10719000491C884010BD1068C00601D50E4810BDBE
:1071A0000E4810BD0E4810BD88020E4B000F185C33
:1071B0000902D368890F491CDB0301D5084A05E0A1
:1071C0001268D20601D5044A00E0044A5043FDF794
:1071D0008FFF10BD0010024000093D000024F400A4
:1071E00000127A00E6A90008FEB505007ED0FE4C2C
:1071F000E7680C20E6680740012000040640287874
:10720000C00747D0082F05D00C2F0AD10120000459
:10721000864206D1206880033CD568680028E5D006
:1072200038E0012069680004814203D121680143EC
:10723000216011E0052301221B0492049942216878
:1072400002D111432160F1E78143216021680140AF
:107250000091206890432060686800280DD0FFF7F7
:107260004BFB009005E0FFF747FB0099401A6428AC
:107270007AD820688003F6D50CE0FFF73DFB00903C
:1072800005E0FFF739FB0099401A6428F0D8206820
:107290008003F6D42878800755D50923E868042FA1
:1072A0000DD00C2F01D1002E09D000283BD0216831
:1072B000994301432160FFF71FFB064627E0216841
:1072C000490701D5002891D061681F22120291431D
:1072D0002A691202114361602168994301432160C8
:1072E000FFF746FFE16809060A0F00E079E1BF49B0
:1072F000895CC840BE4908600020FFF71FFB0028DA
:1073000072D120E0FFF7F8FA801B0228B0D820687D
:107310004007F7D560681F210902884329690902DF
:10732000084360600FE02068400840002060FFF7DD
:10733000E3FA064604E0FFF7DFFA801B022897D83D
:1073400020684007F7D42878C0065FD5002F0CD0FE
:10735000A869002849D02068FF2101310843206036
:10736000FFF7CAFA06462DE0C0E02068800502D586
:10737000A8690028A7D06068072149038843296AC3
:10738000084360606068297F0002000A090608431C
:107390006060286A410B0120C003491C8840E168F5
:1073A00009060A0F9149895CC8409149086000208C
:1073B000FFF7C4FA002817D128E0FFF79DFA801BD9
:1073C0000228A3D820688005F7D560680721490303
:1073D0008843296A084360606068297F0002000AC8
:1073E00009060843606011E0E1E02168FF200130F8
:1073F00081432160FFF780FA064604E0FFF77CFA3C
:10740000801B022872D820688005F7D42878794E2E
:10741000000724D568690028306910D0012108438D
:107420003061FFF769FA009005E0FFF765FA00990F
:10743000401A02285AD830698007F6D50FE0400874
:1074400040003061FFF758FA009005E0FFF754FA6A
:107450000099401A022849D830698007F6D4287864
:10746000400765D500200290A06BC00006D4A06B39
:10747000012109070843A063012002905E480168CA
:10748000C90511D40168821511430160FFF734FA70
:10749000009005E0FFF730FA0099401A642825D8DB
:1074A00055480068C005F5D5FF20AA680130824222
:1074B00003D131690143316111E001218902002AC0
:1074C00007D005231B029A4203D132690A43326175
:1074D000EFE7326982433261306988433061A868DE
:1074E00000280FD0FFF708FA009007E05EE0FFF7F2
:1074F00003FA0099411A4148814257D83069800502
:10750000F5D50DE0FFF7F8F9009006E0FFF7F4F984
:107510000099411A3948814248D830698005F5D42C
:107520000298002804D0A06B012109078843A063BA
:10753000686A002864D00C2F3ED001263606022847
:10754000206805D0B0432060FFF7D6F905462FE04C
:10755000B0432060FFF7D0F9074604E0FFF7CCF90D
:10756000C01B022822D820688001F7D4E96AA86AE3
:10757000E2680843296BFD231B049A431143084327
:10758000E060206830432060FFF7B6F9054604E06C
:10759000FFF7B2F9401B022808D820688001F7D510
:1075A0002EE0FFF7A9F9401B022801D90320FEBDF8
:1075B00020688001F5D423E00128F8D0E06801219B
:1075C0000904AA6A014091420BD10F218904EA6A99
:1075D0000140914205D1032189050840296B884269
:1075E0000ED00120FEBD000000100240D6A9000808
:1075F0001C01002040100240007000408813000071
:107600000020EFE770B5040007D00026254640357E
:10761000A662687C002802D005E0012070BD2E74AF
:10762000204600F02FF8022068742068016840228C
:1076300091430160A168606822690843E1681143D1
:107640000843616901220843A169520211400843BD
:10765000E1690843216A0843A16A08432168086078
:10766000A0690421000C0840616A08432168486051
:107670002068C16992009143C16166650120687408
:10768000002070BD10B586B0044614216846FDF791
:107690008EFD10492068884219D10F48416B821431
:1076A00011434163C16A01221143C162C06A0021D2
:1076B00010400590E02000900220019003200390EC
:1076C00002910491052069460007FFF749F806B0CA
:1076D00010BD00000030014000100240094910B503
:1076E000401E884201D9012010BD074C6061032172
:1076F000081F00F0FFFD0020A0610720206100208E
:1077000010BD0000FFFFFF0000E000E07047704781
:10771000F8B502680446D0691168936805072D0F13
:107720005BD0DD07ED0FFF2621360E402E4367D0DC
:10773000C60706D0CE0504D501261662E26F324395
:10774000E267870702220426002F06DADF0704D04B
:1077500027683A62E76F3743E767470706D5DB07D5
:1077600004D023681E62E36F1343E367020709D561
:1077700020220A402A4305D0236808221A62E36FB8
:107780001343E367E26F002A2FD0800606D58806F0
:1077900004D5216E002901D020468847E06F21687A
:1077A0008968490601D4000724D5204601F0C4FEAB
:1077B00020688168490619D581684022914381601B
:1077C000E06E002812D020498163E06EFEF72EFEA5
:1077D00000280AD0E06E816B06E0850610D58D0684
:1077E0000ED5216E1CE020468847F8BD2046FFF7E5
:1077F0008EFFF8BD2046FFF78AFF0020E067F8BD46
:10780000C50208D55B0206D501200005106220469E
:10781000FFF77CFFF8BD030605D50B0603D5616EA7
:107820000029E0D1F8BD4006FCD54806FAD513681A
:10783000204640218B43136020216167002161664F
:1078400000F069F9F8BD00009594000810B5040037
:1078500003D0606F002802D007E0012010BD002196
:1078600070200155204600F027F82420606720682A
:107870000168490849000160204601F0A7FE01287F
:10788000ECD0606A002802D0204601F0E5FC2068B8
:1078900041680922D20291434160206881682A220E
:1078A00091438160206801680122114301602046F4
:1078B00001F038FD10BD0000F0B587B00646142178
:1078C0006846FDF774FC2C493068884251D12B483A
:1078D000416B0122920311434163C16A01221143AA
:1078E000C162C06A0025104005900320400200904C
:1078F0000220032701A9A1C10420049005206946A4
:107900000007FEF72DFF1F4C1D48A560E56081C4F0
:107910008027E560A7602020256160610002A061EA
:107920001848083CFEF7FCFD002801D0FEF73EF9A0
:10793000F466A662144C12482146143820600320D5
:10794000606010200831A1C16561A561E561204634
:107950002562FEF7E5FD002801D0FEF727F9B466A1
:10796000002201211B20A662FFF734FA1B20FFF73B
:1079700027FA07B0F0BD00000038014000100240B7
:1079800030000240F015002038160020F8B50446FB
:10799000806F20284DD100290BD0002A09D0012367
:1079A000A0681B03984206D12069002803D1C807AC
:1079B00001D00120F8BD25466035287C012838D04B
:1079C000012028745820616502530026E6672220B2
:1079D000A067E06E002819D01749C162E16E174810
:1079E0000863E16E16484863E06E13468663676D70
:1079F00021683A462431E06EFEF7DAFD002805D012
:107A00001020E0672E7420206067D2E72E74206873
:107A10000168FF2201321143016020688168012260
:107A200011438160206881684022114381600020F9
:107A3000F8BD0220F8BD0000F19400082F95000861
:107A4000A994000870477047FFB50446406F83B0A3
:107A500017460D4620285CD1002D0AD0002F08D0F3
:107A6000A168C001814207D12069002804D1E8073C
:107A700002D0012007B0F0BD204660300290007CAB
:107A8000012846D00298012101740020E0672120DE
:107A90006067FEF731FF26464036019037827782D5
:107AA0000120A1680003814202D12069002802D090
:107AB0002F46002511E000270FE0002280212046FC
:107AC00001F098FE002815D1002F15D021683878D4
:107AD00088627F1C708A401E7082708A019B002819
:107AE00006980090E9D100224021204601F082FE54
:107AF000002808D00320BDE728882168C005C00DF4
:107B00008862AD1CE6E720206067029900200874B7
:107B1000B0E70220AEE7704701490248C160FDE7C7
:107B20000400FA0500ED00E010B50524240700224A
:107B300004212046FEF7D9FE002208212046FEF748
:107B4000D4FE0A2002F055F9012204212046FEF756
:107B5000CCFE0A2002F04DF9002204212046FEF757
:107B6000C4FE10BD10B505242407002204212046C0
:107B7000FEF7BBFE012208212046FEF7B6FE0A20D2
:107B800002F037F9012204212046FEF7AEFE0A205A
:107B900002F02FF9002204212046FEF7A6FE10BDB8
:107BA000F8B500240526074625463607002204219D
:107BB0003046FEF79AFE0A2002F01BF9012204214A
:107BC0003046FEF792FE6006040E08213046FEF7AE
:107BD00083FE002801D0641CE4B2052002F009F9FC
:107BE0006D1CEDB2082DE1D3002F03D0FFF79CFFF1
:107BF0002046F8BDFFF7B6FFFAE770B50526054643
:107C00003607002204213046FEF76FFE0024E80903
:107C100001D0012200E0002208213046FEF765FE77
:107C20006806050E0A2002F0E4F80122042130461D
:107C3000FEF75BFE0A2002F0DCF800220421304649
:107C4000FEF753FE0A2002F0D4F8641CE4B2082CBC
:107C5000DDD370BD10B5052424070122082120467C
:107C6000FEF743FE012204212046FEF73EFE0022DD
:107C700008212046FEF739FE0A2002F0BAF8002259
:107C800004212046FEF731FE10BD10B5052424075F
:107C9000002204212046FEF728FE0022082120466B
:107CA000FEF723FE0A2002F0A4F801220421204658
:107CB000FEF71BFE012208212046FEF716FE0A20D1
:107CC00002F097F810BD70B505252D07002401229C
:107CD00008212846FEF709FE062002F08AF8012254
:107CE00004212846FEF701FE062002F082F807E094
:107CF000641CE4B2FA2C03D9FFF7C7FF012070BD62
:107D000008212846FEF7E8FD0028F1D100220421D1
:107D10002846FEF7EAFD002070BD0000F8B501F02E
:107D200031FB01F06BFB46480068C069FEF72EF896
:107D30004449454E898F002914D044490A780121CD
:107D40008902002A0AD0012A04D0022A04D0032A78
:107D500008D103E0212801D2002200E001223046B0
:107D6000FEF7C3FD0121C9023046FEF7B5FD01272C
:107D7000FF03374D0024002825D036480460E879F9
:107D8000002803D10120E87101F078FD28786328EC
:107D900006D9002208213046FEF7A7FD012205E0A2
:107DA000012208213046FEF7A0FD002205203946B9
:107DB0000007FEF79AFD234D274E4035A88C274F2C
:107DC000012803D01CE0EC710022EAE72448694650
:107DD000088072B680212348FDF700FF002804D0F8
:107DE000022269461F48FDF79DFF62B61EA001F002
:107DF000E3FDAC8402F070FD642001F0F3FFFE604F
:107E0000688C012808D10F486C84048002F064FD5E
:107E1000642001F0E7FFFE60288C012806D12C8445
:107E200002F05AFD642001F0DDFFFE600548124AB1
:107E30000188914202D1C088002800D1FE60F8BDBF
:107E400070150020500D0020000400506A00002032
:107E5000D4000020100100200400FA0500ED00E02D
:107E6000AAAA0000384A0008BDF8C8EBC9FDBCB694
:107E7000C4A3CABD0D0A0000AA55000008B53721E9
:107E8000202000F06EF80321212000F06AF8402144
:107E9000222000F066F80821232000F062F8AA21D1
:107EA000302000F05EF80A48008FC1B2322000F0A6
:107EB00058F80221332000F054F85F21202000F010
:107EC00050F8684600F006F80A2001F092FF08BD5D
:107ED000500D002010B501460F2000F021F80028B9
:107EE00000D0012010BD10B50446FFF7B3FE3220CC
:107EF000FFF783FEFFF7E7FEE0B2FFF77EFEFFF736
:107F0000E2FEFFF7A7FE3320FFF777FEFFF7DBFE69
:107F10000020FFF745FE0446FFF7B7FE204610BDE0
:107F200010B50C46FFF7DFFF2070012010BD70B5C3
:107F30000D460446FFF78EFE3220FFF75EFEFFF788
:107F4000C2FEE0B2FFF759FEFFF7BDFE2846FFF77D
:107F500054FEFFF7B8FEFFF798FE0A2001F049FF34
:107F600070BD10B5FFF7E3FF012010BD10B502484A
:107F7000FEF704FE10BD0000E8140020FEB5044624
:107F8000002572B60068394A831804D13849CD6893
:107F9000032189040D4081680191C1680091416904
:107FA0008669002B08D132484038836AC7043B43B6
:107FB0008362836ABB4383620846304348D02B48C0
:107FC0002368C34205D12A48C3680322920493431D
:107FD000C360002917D02068026901231A43026197
:107FE00020684161FEF788FC0746FEF785FC2168A2
:107FF000C01B0968090703D47D21C9008842F4D950
:10800000216808204860002E17D0206801690122ED
:108010001143016120688661FEF76EFC7D270646EC
:10802000FF00FEF769FC2168801B0968C90601D4BE
:10803000B842F6D92168102048600C482168C14236
:1080400006D10B48C1680322920491432943C160C1
:108050002068016949084900016121680198886028
:1080600021680098C86062B6FEBD00000084FFBFB2
:10807000401002401CB5002116480091144A01919D
:108080000260C1631205426081600722826301229F
:1080900002610246C16020321170FF235170C23369
:1080A0004362816211730163816104224163426111
:1080B000C161FEF721F808480090801301906946DD
:1080C0000448FDF7C9FF00210248FDF76FFF1CBD02
:1080D000002401408C1400200200000408B5084868
:1080E000016B012211430163006B012110400090DC
:1080F00000220A20FEF76EFE0A20FEF761FE08BD90
:1081000000100240F0B587B014216846FDF74FF823
:108110004C48C26A04210A43C262C26A0A400592FC
:10812000C16A80273943C162C16A39400591C16A79
:1081300001252943C162C16A29400591C16A02260D
:108140003143C162C06A2A463040059005201C2197
:108150000007FEF7CAFB01223B493C48FEF7C5FB7E
:1081600000223B493948FEF7C0FB9121052000223F
:1081700009020007FEF7B9FB3648019000240520EC
:108180006946009502940007FEF7EAFA0320019081
:1081900005206946009602940007FEF7E1FA0C20DC
:1081A000009011200190032003900520029469465D
:1081B0000007FEF7D5FA10200090052069460396C7
:1081C000019502940007FEF7CBFA1120019002946A
:1081D0006946009503941D48FEF7C2FA1E480190B7
:1081E0006946009602951948FEF7BAFA1B480090B6
:1081F00002946946019503941448FEF7B1FAE80227
:108200006A4651C269461148FEF7AAFA9120000257
:108210000090052002946946019503940007FEF73B
:108220009FFA69460948009702950194FEF798FA6B
:10823000002201210520FEF7CDFD0520FEF7C0FD3F
:1082400007B0F0BD0010024001060000000400501D
:108250000830000000001110000021100836000056
:1082600010B50F4C0D482060FF20053060600020E5
:10827000A060E06020616061E0610121206249024C
:108280006062A161A0620720E0622046FFF7BAF9B0
:108290002068016840221143016010BD0030014098
:1082A0001815002000B585B014216846FCF77FFF43
:1082B0000E480D490160E1214902416000218160C1
:1082C000C160016181610C22C161426101623021A2
:1082D00041620121090381634900C163FFF7B6FAD6
:1082E00001F0C6FA05B000BD00380140701500204D
:1082F000704700008307FF22DB0E9A408907090EB2
:10830000994000280BDA0007000F08388308084856
:108310009B001818C36993430B43C36170478308DC
:1083200004489B001B181868904308431860704766
:1083300000ED00E000E400E0BFF34F8F0449034884
:10834000C860BFF34F8F00BFFDE700000400FA05CF
:1083500000ED00E0FEB50A2002F034F87D20C000F8
:1083600002F04AF8FC4C0025A570A07B0C2801D334
:108370000B20A0730122052051020007FEF7B5FA79
:10838000F648E570F64E00783071F649A079097824
:1083900040000843217D89000843F071E06AF070D5
:1083A000401CE06260793146B0744200B431084646
:1083B000A138FCF7E3FE06207072EB4831460078E6
:1083C000B072207F3073E4481339827F0A75C07F12
:1083D00048756079002240001331153002F0DCF856
:1083E000607900214000153002F0E8F8022002F028
:1083F00039F8F5712574E572012060732573DB4847
:10840000FEF79CFC60840646E5706079FDF736F95E
:10841000D74AD84BFDF72CF801F080FC012300224D
:108420009B07FCF773FFFDF76FF90006C00C80197E
:1084300080B20121C903A084884201D3401AA084DC
:10844000CD48A0632079401C2071C848FEF776FC17
:108450002084C3480C30064642364030019076E115
:10846000C248FEF76BFC2084C44F0BE0BF48FEF708
:1084700065FC81B22184A08C814203D3C04A80185C
:10848000814206D300210F2001F01CFF38422063F7
:10849000ECD0206B411C21D040047DD58122D2013B
:1084A00000210F2002F04DF87D20C00001F0A4FF54
:1084B000002001F056FF0021102001F003FF4106CB
:1084C000A748490E274600225030A16401F030FF32
:1084D000A3485030417A0729C1D101E0FFF72CFFB2
:1084E0000222A849401DFCF76DFE0028B7D102F01A
:1084F000B6F87965386502F09FF8F965B865F878DF
:108500006A46401CF87096484D30017911704079E8
:1085100050701088F98B884274D19B48318A018051
:1085200001988D49808A48839048FEF707FC208493
:1085300001F0DAFDFF23A16D5B04E06D0022C91894
:10854000504100060F0A074379084900080E090246
:10855000216660668248636D0A30226D02F054F82D
:108560006079E36D81007E48A26D0818163002F034
:108570004BF87B48636E1230226E02F045F8784863
:108580000821417260790022800075491C3002F098
:1085900003F86079800000E0CCE000211C3002F09C
:1085A0000DF8384601F007FF012001F05BFF607213
:1085B00002217648FEF790F9002824D0002169486E
:1085C000654A0170B1899186F089D086644F626BEB
:1085D0005037A263FA7C13071B0F032B00D0A37440
:1085E0001209E274012625715B4BE67219875887E0
:1085F000002A16D002226349781DFCF7E3FD00280B
:1086000003D00EE078E00121D9E755482674C67101
:10861000A06C53491638C2B2627466315C48FCF7EC
:10862000ADFD01202073608B5A49FF30C33080B20A
:10863000608388420CD949424018608352480188BF
:10864000491C8AB27D21C90002808A4200D305807C
:108650004D48618B06887D20C00070434018E06360
:1086600002904D48302107784C48E7730088484312
:10867000FCF7E9FF009030460A214843FCF7E3FF8E
:108680000099FCF705FE7F21C905FCF7A8FDFDF761
:1086900003F880B240497F1E0880B84201D1012012
:1086A0002073E6841620205EFCF7D4FF06460F46B2
:1086B000208CFCF7E3FF3A4A3A4BFCF7D9FE0090D6
:1086C00001910298FCF7C6FF019B009AFCF7C2FEDD
:1086D0003B463246FCF71AFEFCF7F2FF2064A08B03
:1086E00000F0A4FC607A002862D100210F2001F084
:1086F000E9FD0006F9D55BE0FDF730FB244A0321D4
:108700000C3A11541449B2898A86F289CA862049E2
:108710008000CC3942180199098B11801C4A796B71
:108720009C3A11500E49FB6D40181630BA6D01F09D
:108730006BFF0CE03A4600210F2001F002FF607948
:10874000E178401C814202D0002001F00AFE208C1A
:10875000A18C884228D283E658000020D400002053
:10876000C41100200C010020E4000020E8140020C7
:10877000B81E85EB51B8CE3FA086010000D027245B
:10878000983A0000F4000020080100200004005086
:1087900074130020E7030000EA000020EE00002030
:1087A000F853E3A59B843E40274A89188842D2D8D3
:1087B00001F09AFC254A00210F2001F0C2FE244856
:1087C0000168A06B3238814208DA214830300068F5
:1087D000002803D0E079401CE07100E0E5711D48FD
:1087E000E27900884100914205D219497839098817
:1087F000E183022121700A2148432179884200D275
:108800002570207C002806D011496C3108784B78FF
:108810008A7802280DD00D4A002180320F2001F005
:1088200090FE01210520002249020007FEF75DF8B5
:10883000FEBD0948C91CC018FCF7A0FC02F04CF8AA
:10884000642001F0CFFA49E6983A000000D02724CE
:1088500008130020E4000020500D002070470000A5
:10886000F0B58DB0B54801900020C0430A900026B5
:108870000A2001F0A7FD7D20C00001F0BDFD002011
:10888000AF4C0546A070AF4FAF480B90AE480022EA
:10889000C23885730146142001F07EFE00211420A9
:1088A00001F08CFE022001F0DDFD00210F2001F01F
:1088B00009FD38422063F8D0206B411C18D04004D9
:1088C0007ED58122D20100210F2001F03AFE002145
:1088D000102001F0F7FC41069B48490E0022801C45
:1088E00001F026FD9848801C417A022902D008E157
:1088F000FFF722FD944802229449C01DFCF762FC58
:108900000028F4D101F0ABFE6165206501F094FE12
:10891000E165A065002E23D10B998D48098A01805D
:1089200089488749801E808A488301268948FEF746
:1089300005FA2084608B8849FF30C33080B26083A1
:1089400088420DD949424018814960830888824A8B
:10895000401C80B20B320880904201D30020088076
:108960000B98694682890A80C0894880764904222A
:10897000C91C0846A238FCF701FCFF22A16D520475
:10898000E06D0023891858410006090A0143084692
:10899000029101F010FD029948084000010E00020A
:1089A000616620666848636D9638226D01F02CFE82
:1089B0006548E36D9238A26D01F026FE624800E042
:1089C000A1E08E38636E226E01F01EFE5E49002229
:1089D000A0393C2001F0E0FD00213C2001F0EEFD3B
:1089E000012001F03FFD6072A0780121401CA070C1
:1089F0000520C9030007FDF7C5F955487D22018808
:108A0000D200084650430291628B0A398018E06315
:108A10000C9052480078E073049008B2208500283A
:108A200003DA7D21C900401820854D483021008897
:108A30004843FCF708FE05902820205EFCF7F8FD6F
:108A40000599FCF725FC7F21C905FCF7C8FBFCF75D
:108A500023FE424980B208800499491E884201D110
:108A6000012020730298E0841620205EFCF7F2FDBE
:108A700005910690208CFCF701FE3A4A3A4BFCF730
:108A8000F7FC079104900C98FCF7E4FD079B049A0F
:108A9000FCF7E0FC059B069AFCF738FCFCF710FE9F
:108AA0002064A08B00F0C2FA00990198814210DA8C
:108AB00000290ED024490422C91C0AA8FCF75EFB39
:108AC0000220207029480A2100784843A0720098AB
:108AD0000190607A002805D100210F2001F0F2FBFF
:108AE0000006F9D5802200210F2001F02AFD002088
:108AF0006D1CEDB26070032D00D2C7E6002E08D0C9
:108B000017E00120F4E71A4A00210F2001F019FDB7
:108B1000F7E7A18B1748002902D00288914201D9BA
:108B20000188A18388B21449401E0988484313492B
:108B300008800A98E0830DB0F0BD00003F420F00AE
:108B40005800002000D0272412120020F40000203A
:108B500008010020E8140020E7030000EA000020DC
:108B6000EE000020F853E3A59B843E40E400002083
:108B700000902724E0000020DE000020DC00002020
:108B8000F8B53B493948086001F046FE2120394CD0
:108B900000016080204640300079374D0006000E0D
:108BA000687003D0E08800280AD00BE07D20C00068
:108BB000E0800120E0870A2060870020A08701E094
:108BC0006420E080208F0A2801D902202087E08ECF
:108BD0003C2801D93C20E086284980B20870E08F0B
:108BE0006871A08FA871A07AE870A68805212E620E
:108BF0006981E7883846FCF77BFAA8810146304650
:108C0000FCF776FA8800081886B27D20C0002E8115
:108C10007043FCF733FD1A4A1A4BFCF791FCFCF742
:108C200073FDE8817D206E823946C000FCF760FA52
:108C300028820146C820FCF75BFA68830120E8829D
:108C4000FDF7A4F8A882EA890F491048FEF77AF8E0
:108C50000FA0296A00F0B0FEE18811A000F0ACFE80
:108C6000218914A000F0A8FEF8BD0000A998000812
:108C700050000020500D0020D400002000000020F3
:108C8000F853E3A59B843E40FF7F0000E8140020DA
:108C9000B1EAC7A949443A202564202E0D0A0000F4
:108CA000CDA8D1B6BCE4B8F43A202564206D732E6B
:108CB0000D0A0000B5A5B4CECDA8D1B6BBF9D5BE7E
:108CC000CAFDC1BF3A202564B8F62E0D0A00000087
:108CD000F0B5924D85B001202880914FC820914C6D
:108CE0003880207A401C2072C00706D0A08B411E1D
:108CF000A183022801D2C820A083A08B00F096F99E
:108D00000A2001F05FFB7D20C00001F075FB02210D
:108D10008548FDF7E1FD002838D000208349800018
:108D20000978844E49000843814909780843B072A4
:108D3000102070728048C1887D20C000FCF7D8F9EF
:108D400070737E487C490078B07330460B308A7867
:108D50000270C9784170411C77482030027ECA7089
:108D6000407E087174482230027E4A71407E8871CC
:108D700000220C39152001F00FFC0021152001F014
:108D80001DFC022001F06EFB6D4E03E00120C5E7E3
:108D9000FEF7C4FF00210F2001F094FA3042206357
:108DA000F6D0206B411C7DD040047CD58122D201BD
:108DB00000210F2001F0C5FB0021102001F082FAF4
:108DC00041065C48490E00225030A16401F0B0FA1F
:108DD000584E5036707A112865D102225949701DBB
:108DE000FCF7F0F900285ED1F01E027969460A709E
:108DF00040794870B17A2980C820FCF779F9388029
:108E0000307BA083504DB01E008A28804549301F1A
:108E1000808A48834D48FDF791FF80B220840390FB
:108E2000608B4B49FF30C33080B2608388420CD9DD
:108E300049424018608328884549401C80B20B3164
:108E40002880884201D3002028802D887D20C00002
:108E5000618B68434018E06302903E4806782846DC
:108E60000A3800B2E6732085002803DA7D21C900A4
:108E700040182085388830214843FCF7E4FB07463A
:108E80002820205EFCF7D4FB3946FCF701FA7F214D
:108E9000C905FCF7A4F9FCF7FFFB2E4980B2088056
:108EA000761E01E037E034E0B04201D101202073AA
:108EB000E5841620205EFCF7CDFB07460191039860
:108EC000FCF7DCFB244A254BFCF7D2FA05460E469C
:108ED0000298FCF7BFFB2A463346FCF7BBFA3A463A
:108EE000019BFCF713FAFCF7EBFB20646846008853
:108EF000E08310480F495030807C6071420063313C
:108F000008465130FCF73AF9A08BFF2801D0032026
:108F1000207005B0F0BDFFF70FFA0000E40000205C
:108F2000EE0000205800002000040050D90000206E
:108F3000DA000020C4110020500D002000000020A5
:108F400000D02724F400002008010020E8140020AD
:108F5000E7030000EA000020F853E3A59B843E40AD
:108F600070B586B014216846FCF721F901250F4E33
:108F7000ED03002229463046FDF7B7FC012000240E
:108F8000019002946946009503943046FDF7E8FB92
:108F90000320019002946946009503943046FDF742
:108FA000DFFB022000F01EFF06B070BD0004005081
:108FB00070470000F8B5044600206A461080194D3D
:108FC00055222A70AA226A700322AA70661DEE70CA
:108FD0002A716971144A49008918AC712246E81D4A
:108FE000FCF7CCF8002007E029186A468978128837
:108FF00089186A461180401CB042F5DB611DA81C2F
:10900000FCF718FD01466846018029190078C871EF
:1090100068464078087221460931024800F0A4FAF7
:10902000F8BD000028140020500D002010B51B4C86
:10903000E18A228A914201D3891AE18289B2628B44
:109040000B4653431B182383132902D14A4310189C
:109050002083208B302148436421643048431049E9
:10906000E0620968401A0F494018A062FCF7F2FA62
:109070000D4A0E4BFCF764FAFCF722FB0C496062C8
:10908000884202DD4A4280186062002801DA4018F6
:10909000606208490968486110BD0000D4000020E2
:1090A00098000020F0D8FFFFF853E3A59B843E40D2
:1090B000FF7F0000E8140020034A1168382389B2BA
:1090C00099430143116070470030014010B5FDF72E
:1090D00019FC10BD10B59AB034216846FCF767F84A
:1090E00014210DA8FCF763F81C2112A8FCF75FF807
:1090F0001B4801680324E402A143C21489180160DB
:10910000FDF774FE17480169A14301610620009034
:10911000FF200130029001200390102004900220D3
:10912000099040040B90000100240C900A946846BA
:10913000FEF75AF80F200D9003200E900F94109414
:10914000012111940DA8FDF73DFF8120129003200D
:1091500080041890149412A8FDF782FE1AB010BD76
:109160000070004040100240104801688215114311
:109170000160C1680E4A1140C16001680D4A11408A
:1091800001608168490849008160016801229204F8
:1091900091430160C168FD2212049143C160002126
:1091A00001610649044888607047000000100240D1
:1091B0000C40FF88F6FFF6FE0050000800ED00E0CE
:1091C00070B501F093F8224C224DE06402E001F00A
:1091D0008DF8E064A842FAD1207801260525F6032F
:1091E0002D07002806D001280CD0022817D003280C
:1091F0002BD128E0012231462846FDF776FBFFF708
:1092000067FD06E0012231462846FDF76EFBFFF7B9
:1092100027FB002231462846FDF767FB15E0A07AC0
:109220000122401EA07231462846FDF75EFBFCF786
:10923000C9FD002231462846FDF757FBA07A0028D9
:1092400003D1207001E0FFF785F800F035FF70BD15
:10925000580000203001CADE10B5818CC90707D044
:1092600001684A6801235B049A43836A1A434A608F
:10927000818C890707D501684A6801231B049A433A
:10928000C36A1A434A60818C490707D501684A6856
:1092900001239B049A43036B1A434A60818C09079C
:1092A00007D501684A680123DB039A43436B1A43DD
:1092B0004A60818CC90607D50268916801231B03A7
:1092C0009943836B19439160818C890607D50168A6
:1092D0008A6801235B039A43C36B1A438A60818CBB
:1092E000490612D503685A6801210905046C8A43AE
:1092F00022435A60026C8A4207D1026851680323F4
:109300005B059943436C19435160818C090607D56D
:1093100001684A680123DB04806C9A4302434A6077
:1093200010BD0000F8B500260446C667FDF7E4FA54
:10933000054620680068124F000709D501212B4619
:10934000002249052046009700F054FA00280DD16C
:109350002068006840070BD501212B4600228905B3
:109360002046009700F046FA002801D00320F8BDFF
:1093700020206067A067603426740020F8BD0000DC
:10938000FFFFFF01F8B5184CC826E078002829D166
:109390006079002826D101206071144D686B002788
:1093A00000281ED0686BC821081A15E01048E16833
:1093B000405C616988470F480A21008848430E498C
:1093C0000880E068401CE060E068C82800DBE760D7
:1093D000696BC820401A761EE168814201D0002ED8
:1093E000E4DC6771F8BD00003C0000200000024092
:1093F000880C0020E4000020F000002070B5224C12
:10940000E07800283FD1207900283CD1012020714C
:109410001E4EF16900250906002933DA21566257EC
:1094200091420AD1F06940062CD5A079002829D0B4
:10943000A5712089401C208124E0A179002903D155
:10944000A0710A2000F0D5FC00202056CC21484312
:109450000F494218206912181279B262401C00228A
:109460002061A256CC235A43895881420ADC2561E7
:109470002078401C207020780E2800D12570A0781C
:10948000401CA070257170BD3C00002000380140D8
:109490006001002010B5806A0022014640314A83F5
:1094A0004A82FEF734F910BD70B5846A606FA56F0B
:1094B0002168896800260906002906DA212804D1D6
:1094C00052200653204600F047F820688068400686
:1094D00006D5222D04D15A200653204600F02CF840
:1094E000E06F10210843E0672046FEF710F970BDD9
:1094F00010B501460968806A0968890614D40022FB
:109500005A210A5201680A68FF2301339A430A600C
:1095100001688A68520852008A6001688A6840239C
:109520009A438A6020218167FEF78CFA10BD10B53E
:10953000806AFEF788FA10BD01680A68FF232133AC
:109540009A430A6001688A68520852008A602021A2
:10955000816700210166704701680A68C0239A4349
:109560000A6020214167704770B5164CE278002AE6
:109570000CD12279002A09D10122E2700025C829E4
:1095800003DC0222A256002A01DCE57070BD012333
:10959000E356CC2253430C4AD1500123E356CC2648
:1095A00073439B180A460146181DFBF7E7FD6078D8
:1095B000401C607060780E2800D16570A078401E55
:1095C000A070E2E73C00002060010020F8B50446EE
:1095D0002669A268E76932436669102000253E4388
:1095E0002368324378491E68784F3E4016431E6018
:1095F00023685A6803263603B243E66832435A604A
:109600002368A2698B4201D0266A32439E680B27E9
:109610003F02BE4316439E606D4E23686D4AB342BF
:109620000CD1D2689207920F06D0012A38D0022AB4
:1096300034D0032A20D11EE001201DE0664EB34243
:109640000AD1D2680C26324026D0042A28D0082A13
:1096500024D00C2A10D10EE08B420DD1D668032203
:109660009202164018D001229202B61A18D0B61AE9
:1096700014D0964200D10820564A0126403A574F4E
:10968000F6038B4236D100280CD002280DD00428D6
:1096900012D008281FD11CE00020EDE70220EBE7E4
:1096A0000420E9E7FDF744FD08E01068C00601D595
:1096B000384605E04A4803E0FDF75AFD002873D01C
:1096C000626851005118814205D81103814202D3CA
:1096D00003E03046F4E7012566E0010E060250087B
:1096E000002330185941FBF719FD03210902411AE3
:1096F0003C4A55E0E169B14232D1030000F083F900
:1097000009070A0D06250606062B0600E3E7FDF706
:109710000FFD1CE0FDF71CFD19E010686168C00634
:1097200002D54808304A01E0304A48088018FBF763
:10973000DFFC80B201462E4A10399142CBD8511C31
:1097400001400007400F08432CE0FDF711FD616860
:1097500040004A08EAE76168012248081204E5E788
:10976000030000F050F909070A0D06260606062C2C
:109770000600B0E7FDF7DCFC1DE0FDF7E9FC1AE0B0
:1097800010686168C00602D54808C01902E0144894
:109790004A081018FBF7ACFC80B20146144A103995
:1097A000914298D82168C8600020206660662846EB
:1097B000F8BDFDF7DDFC61684A088018EAE76168DA
:1097C00048088019E6E7000000480040F369FFEF11
:1097D00000380140401002400044004000093D00B4
:1097E0000024F400FFFC0F0000127A000048E8019A
:1097F000EFFF0000FFB581B017460E4604460A9DF4
:1098000009E0681C07D0FDF777F80499401AA842D0
:109810000CD8002D0AD02068C1693046884318D082
:109820000020B842EDD0002005B0F0BD20680168EE
:10983000FF22A132914301602068816849084900F4
:10984000816020206067A0670020603420740320BE
:10985000EAE70120E5E7000010B504491020096897
:1098600008620248FDF754FF10BD0000701500208B
:1098700001490D20887070473C00002010B5074852
:109880000A22018A51438183FEF728FCFEF70AFD74
:10989000C82203490348FEF779F810BDD400002020
:1098A000880C002070150020F8B53E4C002321786C
:1098B0003D4A1D46082910D0072947D0062950D017
:1098C000052952D0042953D0032954D0002956D059
:1098D000012958D002295AD05BE0A17800264A1FFE
:1098E00004E0314FBF5DFB189BB2761C9642F8DB5B
:1098F000667927799A195118E3786278C918891816
:10990000C9194018C0430006000E1AD1012E14D008
:10991000022E16D125482449C018FBF72FFC00F071
:10992000DBFF642000F05EFABFF34F8F214920482F
:10993000C860BFF34F8F00BFFDE759081046FFF71F
:1099400039FB2570E570A570A571F8BDA17950545B
:10995000491CC8B2A071A178491F8842F5D10820DE
:1099600001E0607007202070F8BDE0700620FAE783
:1099700060710520F7E7A070E5700420F3E7552833
:1099800007D10120EFE7AA2803D10220EBE7032843
:1099900003D02570E570A570F8BD032020702071FC
:1099A000F8BD0000CB000020C4130020500D0020A3
:1099B0000400FA0500ED00E00FB410B503A9044B54
:1099C000044A029800F002F910BC08BC04B0184721
:1099D00021A60008200100202021020C01D0102126
:1099E0001046020A01D010460839020901D010467B
:1099F000091F820801D01046891E420801D0881E26
:109A00007047081A704730B47446641E2578641C89
:109A1000AB4200D21D46635D5B00E31830BC1847C3
:109A200002E008C8121F08C1002AFAD17047704727
:109A3000002001E001C1121F002AFBD1704708B5C8
:109A40000021684601706B46012202212C2000F0A3
:109A500087FD0221684601706B4601222C2000F030
:109A60007FFD08BD38B504466D20694608706B4619
:109A7000012207492E2000F073FD0649002C01D079
:109A8000054A00E0054A2E2000F050FD38BD0000D8
:109A90000608000006180000070600000716000070
:109AA00038B504466B4602220021362000F024FC23
:109AB000B3212300FFF7A7FF0E0F08153A3A3A3AF1
:109AC0001C273A3A2F34483A002168460170407802
:109AD0004108490014E06946087880088000401C6D
:109AE00004E06946087880088000801C08701DE04A
:109AF000684602780A40483202704178802001436B
:109B00006846417012E0684602780A400270407868
:109B10004106490EF4E7694648780221084303E00C
:109B200069464878FD210840694648706B46012225
:109B30000021362000F014FD012200AB1146362032
:109B4000013300F00DFD38BD69460878CF2108408B
:109B500069462030CAE708B50321684641700121F3
:109B600001706B4602220021362000F0F9FC012230
:109B7000D20306212D2000F0D9FC012000F032F99B
:109B80000120FFF78DFF08BD08B5020A69464A703B
:109B900008706B46022204212D2000F0E1FC032016
:109BA000694608706B46012206212D2000F0D8FC82
:109BB0000020694608706B46012206212D2000F026
:109BC000CFFC0A212D2000F07DFB08BDFFB58DB034
:109BD0000446002506E025280AD0109A0F999047E0
:109BE000641C6D1C20780028F5D1284611B0F0BD0A
:109BF00000270121484A009700E00743641C2378AE
:109C00000846203B98401042F7D120782E2817D1E3
:109C1000042007436078641C2A280CD10E98641C29
:109C200002C800910E900BE000990A22514330398E
:109C30004018641C00902078014630390929F3D976
:109C400020780028D1D0642808D0692806D075284B
:109C50001ED0109A0F9990476D1C5BE00A200E9958
:109C6000019001C90E91002802DA40422D2102E044
:109C7000390504D52B216A461172012103E0F90749
:109C800004D02021F7E70BAE0B910DE00021FAE79D
:109C90000A200E99019001C90E91F7E70199FBF78F
:109CA00027FA3031761E31700028F7D103A8801BC7
:109CB00020300190780701D5009801E00120009044
:109CC0000199884201DD401A00E000200027009041
:109CD00006E002A8109AC05D0F9990476D1C7F1C8A
:109CE0000B988742F5DB04E0109A30200F999047DB
:109CF0006D1C0099481E00900029F5DC05E03078C5
:109D0000109A761C0F9990476D1C0199481E01907E
:109D10000029F4DC641C65E709280100F8B54A0055
:109D20002B4B520DD6182B4A0C460546142E2BDA17
:109D3000002E12DA284BFBF7E9FA00221346FBF754
:109D40000FFE40D2002C03DA0124E40700253AE09C
:109D50002046284337D0214C14E0214F0B46F740D2
:109D60003B402B4331D01C4BFBF7D0FA002213466B
:109D7000FBF7F6FD27D2002C03DD01200005F040A3
:109D80000419BC4300251EE0332E1EDC3346002799
:109D9000143BFF43DF40384217D00F4BFBF760FB0B
:109DA00000221346FBF7DCFD0DD2002C0ADD142E39
:109DB0000CD03420811B012088404019A84200D2D9
:109DC000641C0546BD4321462846F8BD641CF9E7DE
:109DD00001FCFFFF9C7500883CE4377E0000F03FEB
:109DE000FFFF0F007D2110B5C900484300F001F8C6
:109DF00010BD002140E000BF00BF00BF00BF00BF9A
:109E000000BF00BF00BF00BF00BF00BF00BF00BF5A
:109E100000BF00BF00BF00BF00BF00BF00BF00BF4A
:109E200000BF00BF00BF00BF00BF00BF00BF00BF3A
:109E300000BF00BF00BF00BF00BF00BF00BF00BF2A
:109E400000BF00BF00BF00BF00BF00BF00BF00BF1A
:109E500000BF00BF00BF00BF00BF00BF00BF00BF0A
:109E600000BF00BF00BF00BF00BF00BF00BF00BFFA
:109E700000BF00BF00BF491C8142BCD37047000037
:109E8000FEB50446002001900090607973494000BF
:109E90000E5A61782578491E7148CFB20163042DAE
:109EA00077D0072D75D000210291217801736C497C
:109EB000E379012292058969002B6CD0914381617D
:109EC0006748217A4173217A82698907890B0A439D
:109ED00082610021042000F034FB324661492E20CB
:109EE00000F024FB3846FFF7BDFD5F4E0522705D94
:109EF000810040185D49431807212B2000F030FBFA
:109F00005B49029801220B180B21282000F028FB46
:109F1000705D584980000A580C21282000F011FB80
:109F2000E079554980004018A1794900425A022140
:109F3000272000F0FBFA51487E00825B0421272095
:109F400000F0F4FAE079002829D0A07804282CD079
:109F500028206946087220220621272000F0E6FA10
:109F600002AB01222621272000F0FAFA44493801E9
:109F70004018E178890042580821272000F0E1FAD2
:109F8000A17A601C627A0902114313D016E000E046
:109F900001E0012188E71143F608816190E764221E
:109FA0000621272000F0C2FAE0E710206946087277
:109FB0000246D1E733490172090A4172417A007AB7
:109FC0000A0202432021272000F0B0FA2E4F0C2174
:109FD00023203A6800F0B5FAF01982880421232082
:109FE00000F0A4FAA07900280BD0E07927490122DB
:109FF00043180021212000F0B3FA03200190012032
:10A0000000902A07120F1001024360780021800798
:10A01000000B0243019800050243009840040243EC
:10A020002079C006400902436079C00602431F2020
:10A0300000F087FAA07861780123084302040848F9
:10A04000DB030261E179490319430A4302610021FC
:10A05000082000F076FA0020FEBD0000A4A9000848
:10A0600024010020042800004CA900080C00002056
:10A070002A00002054A9000874A9000880A900083B
:10A0800084A90008411000006CA900082C000020E1
:10A0900038B50C4607498A8B002102432C2000F07A
:10A0A00045FA684604706B46012206212C2000F018
:10A0B00057FA38BD2401002010B5FFF7C0FC10BDD1
:10A0C00010B504460421362000F0FCF80121C90235
:10A0D000002C01D0084300E08843024604213620CA
:10A0E00000F02FFA10BD000038B540206946087016
:10A0F00000210E2000F0E6F80446002211460E2052
:10A1000000F01FFA6B46012200210D2000F028FA12
:10A11000074A00210F2000F014FA00F0EDF9224662
:10A1200000210E2000F00DFA02480021017338BD15
:10A13000F8FF272444010020FEB5054604206946A7
:10A140000870514C00206075214620312063487111
:10A150000873A0836063A06300F0C8F84B4E2060D2
:10A1600002E000F0C3F82060B042FAD10020FFF70F
:10A1700097FC00F0BBF8464E20603078242801D9C7
:10A18000243806E00621FAF7B3FF0622101A400130
:10A190000843020601040A4301020A430243B26073
:10A1A000706000211E2000F0CCF900F09FF82060C4
:10A1B0006B4601220021242000F0D2F91E20FFF777
:10A1C000E3FC86B2300AA0730420FFF7DDFC0746EB
:10A1D00000F08CF820603806000E0DD00220694691
:10A1E000087101AB012212212D2000F0B9F9A08BDA
:10A1F000012109030843A08300F078F820600620BD
:10A20000FFF7C2FC60600720FFF7BEFCA060F0060D
:10A21000C00E207501D110202075C0B200F0DCF90D
:10A22000E80707D0FFF797FCA08B0121C90208437C
:10A23000A0830AE00521362000F02EF815490840D9
:10A2400002460521362000F071F90120FFF728FCB5
:10A250000021042000F036F8A0610021262000F043
:10A2600031F815218903084302460021262000F019
:10A2700068F900222621362000F058F900F036F85F
:10A2800020600020FEBD0000240100203001CADE55
:10A2900000000020FFFD000038B5094C89B280B2F3
:10A2A0006B46022200F028F8002806D16846407864
:10A2B000010268460078081884B2204638BD0000C4
:10A2C000FFFF000038B50024E44389B280B26B463A
:10A2D000042200F011F8002806D103216846435CEF
:10A2E0002202D418491EFAD5204638BD10B50021E7
:10A2F0000846FFF7E7FF10BD38B5002909D0402414
:10A3000020436C462070C8B27F2906D860700220B6
:10A310000AE069460870012006E0802420436C466C
:10A320006070C809A0700320694600F0AFFA38BD1C
:10A3300010B5144603460A4621461120FFF7DCFFFC
:10A3400010BD10B50346052200211520FFF7D4FFEC
:10A3500010BD10B50346052200211720FFF7CCFFE2
:10A3600010BD38B5054600206946087000F0C4F8F5
:10A37000FF2401342246002D01D0032212020021C5
:10A380000D2000F0D3F8002D13D06B4601220321DD
:10A390000F20FFF7B1FF68460078000709D5FFF7E7
:10A3A000A3FE224600210D2000F0C0F80020C0438B
:10A3B00038BD002038BD10B5024601210A2000F04A
:10A3C000C0F810BD10B5044600211A20FFF77AFF2F
:10A3D000000D22030005120B024300211A2000F099
:10A3E000B0F810BD10B5024602492E2000F09EF8CC
:10A3F00010BD000004180000F8B505466B460122A8
:10A4000003210420FFF778FF0126114C3607002DA9
:10A410000DD02A4600210C2000F088F86946087803
:10A420001021084369460870A069304307E0694677
:10A430000878EF21084069460870A069B0430B46D0
:10A44000A06101220321042000F08AF8F8BD000079
:10A450002401002010B502460021182000F066F803
:10A4600010BD0000F8B50746002568460570B8071E
:10A47000204C2E4600280ADA8020694608706B4678
:10A48000012200210D2000F06BF801202073F80755
:10A490006946087821D006210843694608706B4652
:10A4A000012200210D2000F05BF803210F20FFF7AF
:10A4B000F3FE8121C900084219D040206946087086
:10A4C0006B46012200210D2000F04AF80020FFF722
:10A4D000F7FD00252673ED4309E002210843694694
:10A4E00008706B46012200210D2000F039F8284643
:10A4F000F8BD0000440100201CB56B460122032179
:10A500000F20FFF7F9FE684600784022C10910408D
:10A51000C9014000814208D0012069460871024605
:10A5200001AB03210D2000F01BF81CBD08B56B46E4
:10A530001A70120A5A7089B280B2022200F010F822
:10A5400008BD38B500236C46E254120A5B1C042B8C
:10A55000FADB89B280B22346042200F001F838BD4C
:10A5600038B58024002909D0C02528436D462870BD
:10A57000C8B27F2907D86870022009E020436946E5
:10A580000870012004E020436870C809A870032007
:10A59000694600F0B7F938BD10B51446012312180A
:10A5A0009B029A4202D90020C04310BD0B46821E76
:10A5B00021460920FFF7D4FF002010BD10B5054A41
:10A5C0008905126901430A4300210820FFF7B9FFFA
:10A5D000002010BD2401002038B504466B4601223E
:10A5E0000E212B20FFF788FE68460078E10640091F
:10A5F0004001C90E0143684601706B4601220E21DD
:10A600002B20FFF7ADFF38BD10B5002142541C06CA
:10A61000120A22431B0A491C0429F7DB10BD000063
:10A6200013B501231A4669460248FDF70DFA009852
:10A630001CBD0000701500207CB50024254668462E
:10A64000FFF77FFE04206946220E2D0215432202E9
:10A650000C5C1443401EF7D5204629467CBD7CB5D2
:10A66000002425466846FFF774FE04206946220E42
:10A670002D02154322020C5C1443401EF7D52046E0
:10A6800029467CBDFCF746F9FEF724FDFDF73AFDAF
:10A690003C493D48002522C005608561C5613B49B4
:10A6A0000562C1600838FCF7CFFAFDF717FDFDF72A
:10A6B000F9FDFDF7D5FDFDF7DDFC05260122360786
:10A6C000D1033046FCF711F9FEF75AFAFDF7D6FB35
:10A6D000FBF710FAFBF7DEF90721B015FFF7D8FCFE
:10A6E0002B4C0A21208A01224843A08317033946B4
:10A6F0003046FCF7FAF82448C82226498830FDF78E
:10A7000045F9254E2079002839D06078002836D0C8
:10A71000FEF7E0FC2571FBF7D5FB20700F2809D967
:10A72000012239463046FCF7E0F8FEF749FD0022E9
:10A73000394609E0012251033046FCF7D6F8FEF70E
:10A740003FFD0022012149033046FCF7CEF8FDF71A
:10A75000E5FAA08B002801D0401EA0830F48A18BF2
:10A7600000780843CED10121C9023046FCF7B4F885
:10A770000028C7D101210846FCF758FBC2E7FDF7C6
:10A78000CDFABFE7007C0040E8140020FFFF000086
:10A79000D4000020880C002000040050420000205B
:10A7A00010B586B01748FCF7D4F914216846FAF7BB
:10A7B000FEFC154800900320019000200290052027
:10A7C00069460007FBF7CCFF69461048FBF7C8FF56
:10A7D00069460F48FBF7C4FF01210846FCF726FB3A
:10A7E000FF2401342046FCF7F9FA0A4908680422DC
:10A7F000104308602046FCF701FBFCF707FB06B09E
:10A8000010BD0000E8140020FFFF0000000400500D
:10A81000000800500070004010B501229202184953
:10A820001848FBF7F5F91648174902888A4226D0DE
:10A8300001807D21C90081804910C1800A210181E8
:10A8400000211E224181D24382810122C2810184E2
:10A85000018241828182C182018381831E23C3865A
:10A8600002230387782343878287C28702464032C8
:10A87000118451849184C183918000F02DF810BD22
:10A88000500D002000FC0008AA550000F0B58C46D1
:10A8900000251026052109078E620E4C08E0674648
:10A8A0007F5DE760A768FF07FCD0E7681F706D1C3D
:10A8B0008542F4DB0020074606E0E760A568ED0767
:10A8C000FCD0E5681D54401C9042F6D38E610020F8
:10A8D000F0BD00000030014070B572B60124074D94
:10A8E000A40221462846FBF779F9002804D0224625
:10A8F00003492846FBF716FA62B670BD00FC000853
:10A90000500D0020F0B50025102605279C463F0776
:10A910000B46BE620C4C06E0595DE160A168C907B8
:10A92000FCD0E1686D1C8542F6DB002007E0614643
:10A93000095CE160A168C907FCD0E168401C904255
:10A94000F5D3BE610020F0BD0030014000000102DF
:10A9500003040005405C0000A05C0400C06C08001B
:10A96000805C0400E03F1E00E07D1E0007A9022578
:10A9700070889B880A001600010006000100020092
:10A9800087008D002D001A3152001A339A001A35B3
:10A990001D011A376B003B31BE003B335E013B3576
:10A9A00096023B37000099599959EB518F421E4549
:10A9B000142E0080EB51F5283333E13A703DE13A33
:10A9C000C235852BC2353333C235C235AE47E13A85
:10A9D0005138A3305138000000000000000001028F
:10A9E000030406070809030406080C1018203000A9
:10A9F000000000010203040018AA00080000002063
:10AA000024010000209A00083CAB0008240100202B
:10AA100074190000309A00080000000000000000D7
:10AA200000000000070400091E0805400826091060
:10AA300040085608054008261D040008BE1D0400F5
:10AA400008BED8BC40100800010000000000C84249
:10AA500000000000000000000000000000000000F6
:10AA600000000000000000000000000000000000E6
:10AA700000000000000000000000000000000000D6
:10AA80000000000000005C12000000000000000058
:10AA900000000000000000000000000000000000B6
:10AAA00000000000000000000000000000000000A6
:10AAB0000000000000000000000000000000000096
:10AAC0000000000000000000000000000000000086
:10AAD0000000000000000000020204000909010259
:10AAE00000810000000000000100000000000000E4
:10AAF0000000000000000000000000000000000056
:10AB00000000000000000000000000000000000045
:10AB10000000000000000000000000000000000035
:10AB20000000000000000000000000000000000025
:0CAB3000000000000000200000000000F9
:04000005080050C1DE
:00000001FF
